:100000000020001003010000D5000000D700000010
:1000100000000000000000000000000000000000E0
:10002000000000000000000000000000D9000000F7
:100030000000000000000000DB0000003D0E00009A
:10004000DF000000DF000000000000008D0D000058
:10005000DF000000DF0000000000000000000000E2
:10006000DF000000DF000000DF000000DF00000014
:10007000DF000000DF00000000000000DF000000E3
:100080000000000000000000000000000000000070
:100090000000000000000000000000000000000060
:1000A000DF000000E504000005050000DF0000009F
:1000B000DF000000DF000000DF000000DF000000C4
:1000C000F81D0000000000100000000000000010FB
:1000D000AC020000FEE7FEE7FEE7FEE7FEE7FEE714
:1000E000002310B5934203D21C585C500433F9E747
:1000F00010BD00238B4203D200221A500433F9E7CB
:100100007047882370B5104E104D114C33602B6032
:10011000104B9C4206D220686168A268FFF7E0FF9E
:100120000C34F5E70C4B9C4205D220686168FFF760
:10013000E0FF0834F6E7882333602B6000F0B0FD61
:1001400001F098FBFEE7C046584004405C40044084
:10015000C0000000CC000000D4000000FFFFFFFF43
:10016000FFFFFFFFFFFFFFFFFFFFFFFFFFFFFFFF9F
:10017000FFFFFFFFFFFFFFFFFFFFFFFFFFFFFFFF8F
:10018000FFFFFFFFFFFFFFFFFFFFFFFFFFFFFFFF7F
:10019000FFFFFFFFFFFFFFFFFFFFFFFFFFFFFFFF6F
:1001A000FFFFFFFFFFFFFFFFFFFFFFFFFFFFFFFF5F
:1001B000FFFFFFFFFFFFFFFFFFFFFFFFFFFFFFFF4F
:1001C000FFFFFFFFFFFFFFFFFFFFFFFFFFFFFFFF3F
:1001D000FFFFFFFFFFFFFFFFFFFFFFFFFFFFFFFF2F
:1001E000FFFFFFFFFFFFFFFFFFFFFFFFFFFFFFFF1F
:1001F000FFFFFFFFFFFFFFFFFFFFFFFFFFFFFFFF0F
:10020000FFFFFFFFFFFFFFFFFFFFFFFFFFFFFFFFFE
:10021000FFFFFFFFFFFFFFFFFFFFFFFFFFFFFFFFEE
:10022000FFFFFFFFFFFFFFFFFFFFFFFFFFFFFFFFDE
:10023000FFFFFFFFFFFFFFFFFFFFFFFFFFFFFFFFCE
:10024000FFFFFFFFFFFFFFFFFFFFFFFFFFFFFFFFBE
:10025000FFFFFFFFFFFFFFFFFFFFFFFFFFFFFFFFAE
:10026000FFFFFFFFFFFFFFFFFFFFFFFFFFFFFFFF9E
:10027000FFFFFFFFFFFFFFFFFFFFFFFFFFFFFFFF8E
:10028000FFFFFFFFFFFFFFFFFFFFFFFFFFFFFFFF7E
:10029000FFFFFFFFFFFFFFFFFFFFFFFFFFFFFFFF6E
:1002A000FFFFFFFFFFFFFFFFFFFFFFFFFFFFFFFF5E
:1002B000FFFFFFFFFFFFFFFFFFFFFFFFFFFFFFFF4E
:1002C000FFFFFFFFFFFFFFFFFFFFFFFFFFFFFFFF3E
:1002D000FFFFFFFFFFFFFFFFFFFFFFFFFFFFFFFF2E
:1002E000FFFFFFFFFFFFFFFFFFFFFFFFFFFFFFFF1E
:1002F000FFFFFFFFFFFFFFFFFFFFFFFFFFFFFFFF0E
:100300000823802230B5041C1440651EAC4149000E
:100310000919064C5208A14202D9054C89B2614024
:10032000013B002BEFD188B230BDC046FFFF00007B
:100330002110000070B50E1C051C041C0021331B8D
:10034000EB18002B05DD2078FFF7DAFF0134011CE4
:10035000F5E70020FFF7D4FF011C0020FFF7D0FFD6
:1003600070BD000038B529480F21002201F03AF88D
:1003700026481021002201F035F8244812210022DD
:1003800001F030F821481921002201F02BF81F4814
:100390001A21002201F026F81D48002101F074F90D
:1003A0001B4801F087F91A4D2B685B00FBD400F065
:1003B000EDFE184901F065FAFF232C680138C0B240
:1003C0009C43154904432C60CA6F144B14481340D6
:1003D00080221343CB67E023124A5B00D4582040AD
:1003E000D050D45810482040D050D4580F48204006
:1003F000D050D4580E482040D050D4580D482040FA
:10040000D050CA6F0C4B1340CB6738BD004004403E
:1004100000C0014080C3C90104800440FFFFEF25F4
:10042000FFDFFF0100C00040FFBFFF01FF7FFF01B2
:10043000FFFFFE01FFFFFD017FFFEF25012280236B
:10044000824030B58025DB021A430F4B2D069A609F
:100450009C680E4A14402C439C609C682240802477
:10046000E40422439A60021C083292009A58940FC6
:10047000F9D0002902D01204120D0A809968044AAA
:100480000A409A6030BDC04600C00140FF7F0CFCAE
:10049000FF7F0C7C7FB5482301AA0838517010708B
:1004A00002A902208B730023088104488B814B81B1
:1004B00002924B6001F0A4F907B000BD00000540B6
:1004C000012808D002280BD1A02300221B065A764F
:1004D0000132DA7604E0A02300221B069A76187413
:1004E000704700000223054A5362054A1380A02387
:1004F00000221B069A7601321A747047004000A051
:10050000000000100422064B5A62064B023A5A8041
:10051000A02300221B065A760132DA767047C046C5
:10052000004000A000000010F8B50227354BA024C1
:100530001F805F8080228E2324069B015202E2509E
:10054000802180228020C90480041205E250E150FD
:10055000E050BE2318222C4D5B00EA50093A0433C8
:10056000EA50902380229B015204E2508022120222
:10057000E250FD22254B1E6832401A60FB225F616B
:100580001E6832401A600422214E5A61AD18306054
:1005900002C6EA6F1F4B2049134080221343EB67CA
:1005A000E0231E4A5B00D0580140D150D0581C496E
:1005B0000140D1501B483A1C082100F01DFF3A1C95
:1005C0000721184800F018FFEA6F174B1340EB673C
:1005D000164D281C00F030FD2723281C6B611449A0
:1005E00001F08AF81E232A681340012213432B606E
:1005F00080235B00F3670023A37622746376E276A0
:10060000F8BDC0460000001000800440004000A07B
:1006100000E100E0FFFFEF25FFF7FF0100C0004011
:10062000FFEFFF01004004407FFFEF250000054081
:10063000A086010070B50C1C002827D001284CD1E1
:100640000AB2A02300211B068A421CDAFA2619747A
:10065000B600A0252D062B7E002B04D00123214AB5
:10066000AB7613800BE00120013E00F079F9002EFB
:10067000EFD101230222AE762B741A4B1A808F2100
:100680000020214023E09976187426E0A0230AB2C6
:100690001B06002A1EDAFA26D876B600A0252D06FB
:1006A000EB7B002B04D001230E4A6B7653800BE0CA
:1006B0000120013E00F054F9002EEFD10123022267
:1006C0006E76EB76074B5A808F2101202140FFF791
:1006D000E1FE02E001225876DA76322000F04CF991
:1006E000002070BD00000010031C0120834203D8CD
:1006F000C01A024B4000185C7047C0460000001052
:100700003A2330B58BB00093041C05A96846174BFB
:100710009847059D0120002D26D1069B201C1A0C10
:1007200019069BB2090C1B0A0B43110A1206120C84
:100730000A431B04134306A90422069301F092F80E
:10074000079B201D1A0C19069BB2090C1B0A0B43B0
:10075000110A1206120C0A431B04134307A90422B0
:10076000079301F07FF8281C0BB030BDF11FFF1F6D
:10077000A021054B09061A780020002A00D101208B
:10078000D24308731A70704704000010A021054B73
:1007900009061A780020002A00D10120D2434872AD
:1007A0001A7070470C000010A021054B09061A783A
:1007B0000020002A00D10120D24308721A7070472D
:1007C00012000010A021054B09061A780020002A0B
:1007D00000D10120D24348731A70704713000010F3
:1007E00010B58E23A024802224069B019201E250A2
:1007F00080225201E25080229200E250013AFF3AF8
:10080000E250FA2000238000637323736372237223
:1008100000F0A6F80123637323736372237210BD83
:1008200070B5061E43D0012800D07FE0404D414CFA
:10083000298002230A0709D5FA21226803201343DD
:1008400049003D4A236000F04BFB08E0226803208A
:100850009A43226000F054FBA0231B061E732B88D2
:1008600001265B0709D5FA21236802201E434900AF
:10087000324A266000F034FB08E023680220B343CC
:10088000236000F03DFBA0231B065E73A023298894
:100890001B060122880702D50020187300E01A7396
:1008A000114201D0002200E001225A733EE00823E9
:1008B0001F4D204C69802268194208D0FA21134349
:1008C000052049001E4A236000F00AFB08E09A4315
:1008D0000520226000F014FBA02301221B061A72DF
:1008E00004206B88034208D0FA212368490003439F
:1008F000144A236000F0F4FA08E02368834323607D
:1009000000F0FEFAA02301221B065A72A023698878
:100910001B060122880702D50020187200E01A7217
:10092000114201D0002200E001225A7270BDC0467F
:100930000E0000100800001071070000C50700003D
:10094000A90700008D0700000023012804D8013307
:10095000181A9840014BC35A181C70470E0000101B
:10096000002806D0034B0138C046013B002BFBD1C9
:10097000F6E77047B80B0000002804D00138C046E5
:10098000C046C046F8E77047F0B587B000F040FDBC
:1009900000F026FBFFF7C8FD00F070FAFFF720FF1C
:1009A000FFF7E0FC00F080F90020B449021C00F0E1
:1009B00097FAFA2101208900002200F091FA002420
:1009C000012C00D1E1E000F0EFF9272800D8D7E0B2
:1009D000AB4D00212822281C00F048FF281C2821AC
:1009E00000F0EAF90024061E282E00D0D5E0EB1D09
:1009F000DF7F2B1C0833DB7F3F02A81D20211F4314
:100A0000FFF798FC874200D0BAE0201C9B49221CCB
:100A100000F066FAAB78242B00D197E00CD8102BAD
:100A200018D0222B00D0ABE0A979EB790902287904
:100A30001943FFF7FFFDA3E0282B00D191E0302BF5
:100A400000D09DE08F4D321C281C211C00F00EFFB1
:100A50002E1C2BE08B4D211C321C281C00F006FFA5
:100A6000AF1D8948FFF74CFE87490822381C00F06B
:100A7000F9FE281C0F2285490E3000F0F3FE4323B7
:100A80002B700B336B700E3BAB703F3B2B716B715C
:100A90002021EC70381CFFF74DFCEB1D020ADA77C1
:100AA0002B1C0833D877311C281C4CE0784BE25AB9
:100AB0003319110A02349971DA710A2CF6D1002423
:100AC0000020FFF711FE201C2C74FFF70DFE687448
:100AD0000120FFF709FE0120AC74FFF705FEE87462
:100AE000201CFFF731FF000A2875201CFFF72CFFA0
:100AF00068750120FFF728FF000AA8750120FFF79D
:100B000023FF0121634BE87559561A8829766A76C6
:100B10005A88DB7820215BB2AB7643232B700B33F2
:100B20006B70063BAB70473B2B716B71EC70B01D6B
:100B3000EA76FFF7FFFBF31D020ADA77331C08336E
:100B4000D8772821301C00F06BF919E0EB78002BE6
:100B500016D1A979EB79090228791943FFF760FECC
:100B60000EE02979AB79EA79012909D81B021343F0
:100B70001AB2002A04DA1B05464A49001B0D8B52A3
:100B8000002000F0C9F9041C07E000F00DF9002472
:100B9000272383426441E4B230BF012000F0BCF956
:100BA000002800D10CE73C4E3C4D31880320033136
:100BB00049006918FFF742FC318804204900691890
:100BC000FFF73CFC31880120063149006918FFF726
:100BD00035FC318802200C3149006918FFF72EFCE2
:100BE00031880020093149006918FFF727FC328855
:100BF0000023013292B2022A01D8328000E0338011
:100C0000002201AE01937360B360F360336100238F
:100C1000062159439F00A818415AF0590133091879
:100C2000F151052BF4D10232062AF0D100277B00C6
:100C3000F058032100F025FE00F0CEFE00F088FE03
:100C4000134D785302370A2FF1D1124E6A880221D0
:100C5000735E9A4202DC0120FFF732FC2A880021F1
:100C6000735E9A4202DC0220FFF72AFCFA2101207F
:100C70008900002200F034F9A2E6C046B80B00005B
:100C80006E0000101C000010140000104A1A000032
:100C900062000010960000106C000010440000106C
:100CA00008B500F0C3F908BD2B4A70B5141DE16FFB
:100CB0002A4B01250B408021802629480B434131D6
:100CC000E367FF3143587604DB01DB092B434350D4
:100CD00043589432DB01DB0933434350BD3915607F
:100CE0000020FF3900F06AFB281C002100F066FBA1
:100CF000E26F1C4B04261340E3671B4C201C00F0E2
:100D0000B1FAE1202268194B291C134033432360B8
:100D1000400300F06BFAE121201C490200F0EAFADE
:100D20002268134B134913402B4323606268124B14
:100D30001248134063602A1CA02300F087FB2A1C82
:100D40000F49A0230F4800F081FB08220E4BE560FD
:100D500026611A6070BDC04600800440FFFFEF2589
:100D600000C000407FFFEF250040064001DAFC0094
:100D70007CDAFC009A000010060301003C01001020
:100D8000640100105001001000E100E008B50348C4
:100D90000349044A00F0FCFA08BDC0460040064082
:100DA0003C01001050010010024AD3681069181A63
:100DB0007047C0463C010010F0B585B002AB9D1DE8
:100DC000002302AA144ED71D01912B703B70041C06
:100DD00001331248311C2A1C00F0D3FA2B78432B24
:100DE00001D0002016E001230C48311C3A1C00F011
:100DF000C8FA3B784E2BF4D1201E0AD02A786370B3
:100E0000019B2270023BA21C0448311C00F0B9FA7D
:100E100080B2023005B0F0BD3C0100100040064039
:100E200008B5021E04D00B1C0248034900F08EFADC
:100E300008BDC046004006405001001038B50D4CBA
:100E40000D4D231F1B78002B0FD02368002B0CD0D7
:100E5000013B2360002B08D1A368002B01D09847E9
:100E600001E001232373636823601434AC42E8D1AA
:100E700038BDC0460C020010AC02001010B5124B79
:100E8000124A0024191F0C701C605C609C601C736B
:100E900014339342F5D1FA210D4B8900186800F004
:100EA000F0FC0C4B013898420CD80B4A0B495060AF
:100EB000C0200B6A00061B021B0A03430B620723B8
:100EC0009460136010BDC0460C020010AC0200100C
:100ED000A8020010FFFFFF0010E000E000ED00E0BE
:100EE0001423584310B5054C133B03550023201819
:100EF00041608160C260037410BDC04608020010EA
:100F000014235843034A835C002B01D000238354ED
:100F10007047C046080200101422131C43430349C3
:100F2000585C002801D0CB18187C704708020010CC
:100F3000234A38B5141DE16F224B80250B408021D8
:100F400021480B434131E367FF314358AD03DB01D7
:100F5000DB092B43802543504358ED03DB01DB09BC
:100F60002B4343500125112094321560011C00F0E1
:100F700025FA1220011C00F021FAE26F134B1340F6
:100F8000E367134C201C00F06DF92268114BE1203F
:100F90001340042213432360291C400300F026F968
:100FA000E121201C490200F0A5F921680A4B1940F3
:100FB000294321606268094B1340636038BDC04615
:100FC00000800440FFFFEF2500C000407FFFEF25B9
:100FD0000080064001DAFC007CDAFC000603010018
:100FE00010B5A0242406FFF7A3FF201C00F018FA78
:100FF0008E22802392019B028021A350012349026B
:101000006374A150802109052374A150E37610BDBB
:10101000044A054BD16F0B408021C9020B43D367B3
:101020007047C04604800440FFFFEF2508B5FFF776
:10103000EFFF00F001FA08BD30B5184C1622A042AF
:1010400008D0174B0132984204D0164B023A98420E
:1010500000D0103A01219140134D144AEB6F134018
:101060000B43EB670F22A04208D00D4B0132984290
:1010700004D00C4B023A984200D0083A0123934026
:10108000181C0B490B4B4C6803439C434C604B684A
:10109000094A134003434B6030BDC046000007407F
:1010A000004007400040054004800440FFFFEF255A
:1010B000008004400020FEFFFFDF01000022034B00
:1010C00018645A6401325A647047C0460080044074
:1010D0000022034B18675A6701325A677047C046AF
:1010E0000080044008B5074B596A1F23CA05120F38
:1010F0001940054B920001314900D05800F0C1FB66
:1011000008BDC04600800440641A0000084B1A6CF9
:1011100003231340012B06D0032B06D00020002B05
:1011200005D1044803E0044B00E0044B1868704705
:1011300000800440001BB7005C1A0000601A000029
:10114000044B10B59C68FFF7E1FF1F2323400133D8
:10115000584310BD0080044008B50A4B1A6F0323A2
:101160001340022B06D0032B07D0012B08D1FFF729
:10117000CDFF06E0FFF7B6FF03E0FFF7E1FF00E079
:10118000014808BD00800440001BB70008B5FFF708
:10119000E3FF034B996FC9B200F073FB08BDC04673
:1011A0000080044038B50020FF240D4B1D68254009
:1011B000854213D0FFF7D0FF291C00F062FB094BDA
:1011C0001A681440FF2C09D1074B010E1A6800025F
:1011D0001440621CFF32002300F08CFB38BDC04677
:1011E00094800440F0800440F4800440F8B5051C6D
:1011F0000F1CFFF7B1FF291C061C00F042FB011E6B
:1012000000D10131FF24081C104B20401860104A07
:101210001048002F15D057680F4B3B40536057685C
:101220000E4B3B4004273B4353600460301C00F0EE
:1012300028FB291C000200F024FB094B04401C6021
:1012400000E00760FFF7AEFFF8BDC04694800440A1
:1012500000800440F0800440FBDF0100FFDF01005C
:10126000F480044070B5194C0E21A04205D0184BF3
:10127000C1184A4251411023591A01258D40154E7B
:101280001549F26F154B0A402A43F267144AA042EF
:1012900007D1586813490140596059680A4008212C
:1012A00011E01149884207D158681049014059603E
:1012B00059680A40102106E058680D4901405960FC
:1012C00059680A4020210A435A6070BD0040064018
:1012D0000080F9BF04800440FFFFEF250080044038
:1012E000FFDF0100F7DF010000800640EFDF0100B3
:1012F000DFDF010038B50C1C051CFFF753FF21018F
:1013000000F0BFFA0138286238BD37B5041C0D1C47
:10131000A368DB0707D56A466369D11D281C0B70DB
:1013200000F09CF8F4E737BD73B5051C0E1CAB68E4
:101330005B070AD56B46DC1D301C211C00F0ECF865
:10134000002802D02378EB61F1E773BDF7B5019374
:101350000423061C0F1C151C0361081C111C019A98
:1013600000F097F8041C391C301CFFF7DDFF019BCF
:1013700029191A1B381C00F08CF804230019F3609B
:10138000FEBD08B5081C111C1A1C00F0DEF808BDD3
:10139000F8B504268368041C0F1C151C334207D0C3
:1013A000111CFFF7C1FFEA682B699A4200D1266140
:1013B000391C201CFFF7A9FFF8BD00000F2310B552
:1013C000FF240340DB009C40054A00098000801890
:1013D00002689940A243131C0B43036010BDC04632
:1013E00000C000408900411818200B68D2008343D8
:1013F0001A430A6070470000890041180868034BCF
:10140000120203401A430A607047C046FFFCFFFF08
:1014100008B5FFF7BBFE014B186008BDA80200101D
:10142000034A044BD16F0B4040210B43D3677047F5
:1014300004800440FFFFEF2508B50248024900F090
:10144000C7F808BD0087930380C3C9014360002328
:10145000016082600361C36001207047F8B5041C1D
:10146000C3680768626800691B1A002093420FDA9C
:101470000D1CE068111C00F004FAA6687143321CD0
:101480007818291C00F0EEF90120E3680133E360CD
:10149000F8BDF7B5036846680193C36804691C1B6F
:1014A0000023B44236DAC36807690091041C311C7A
:1014B000C068DF1B151C00F0E4F9F71B7B18381C13
:1014C000B34200D3701A3F1A061EAE4200DD2E1C36
:1014D000AD1BBD4200DD3D1CA268019B5143724320
:1014E0005818009900F0BEF9E3686168F018E060F0
:1014F00000F0C7F9A768236879435818391C3A1CCB
:101500007143009B6A43591800F0ACF9E3685B191A
:10151000E3607319181CFEBDF8B5C2680369041CAA
:10152000076800209A420FD00D1C2069616800F006
:10153000A8F9A668281C7143321C791800F092F9AA
:101540000120236901332361F8BDF7B50368C4683E
:101550000193036900269C4238D04668C768036936
:101560000091041C311C0069FF1A151C00F089F958
:101570007B18381CB34200D3701A3F1A061EAE42C5
:1015800000DD2E1CAD1BBD4200DD3D1CA268019B91
:10159000514300987243591800F064F9A768236911
:1015A000391C7143F018009B20615B18616800933F
:1015B00000F067F93A1C794323686A435918009888
:1015C00000F050F9236976195B192361301CFEBDC8
:1015D000F8B5051C081C274900F053F90024061E25
:1015E0001E2E45D8281C234900F04BF960283FD80F
:1015F000251C0C246C43204F83B2E25B9A4224D119
:101600003C196288B3B29A421FD11C4B02201D8044
:1016100000F016F90020FFF751FD0020FFF758FDFC
:10162000174B80201A6901221A6100F0F9F8032390
:101630001F22218980200B405901E388114C13405F
:101640000B43A36000F0FCF804E00135472DD0D136
:1016500000240DE00126E3683342FBD00C246C43E8
:101660003F197A89074B03209A67FFF731FD341C35
:10167000201CF8BD40420F00A41A00000402001014
:10168000000004400080044038B5041C10200D1CEC
:1016900000F0D6F8054A064BD16F0B408021490473
:1016A0000B43D36700236366256038BD0480044084
:1016B000FFFFEF25802238B50368D205134303608E
:1016C00002680A4B041C13400360FFF75FFD0849E2
:1016D00000F0D7F8FF2325680138C0B29D430543C9
:1016E00025602268034B1340236038BDFFFEFFFFD7
:1016F00020A10700FFFBFFFF38B5041C0D1CFFF7FE
:1017000045FD616989B20131694300F0BAF84208C8
:1017100092B2801A80B20223012A04D9131C092A2A
:1017200000D909239BB20222012804D9021C0928EE
:1017300000D9092292B2023B023A1B0113436362B1
:1017400038BD1022031C406810B5104201D005209E
:1017500003E04022104203D0032088815A603BE01E
:101760000122104237D058680007400F042832D8B1
:1017700000F063F90306122A2E000122DA602BE042
:101780004A68501C4860986A10704A89013A92B2BF
:101790004A81002A19D009E00A89002A08D008687D
:1017A000013A441C0C60007898620A81012209E029
:1017B0004A89002A09D001208A7B52000243D2B212
:1017C0009A6202221A6207E002228A810422F9E761
:1017D00004228A81F6E78A818889FF38431E98416E
:1017E00010BDFF238B81AF3B43608B7B5A000B897D
:1017F00059424B411343DBB28362022303627047B9
:1018000038B5041C0D1CFFF7ECFF6368DB07FCD543
:10181000201C291CFFF795FF0028F6D038BD0000DA
:101820008E22054992008B581843044B1840DA2346
:10183000DB0118438850704700800440FF8000009F
:101840008E2110B5054C89006358054A13400240AB
:101850009343DA22D2011343635010BD0080044049
:10186000FF80000008B500F0BDF808BD08B500F025
:10187000CFF808BD08B5FFF787F808BD03000B4394
:1018800021D4002931D00122D207030901E0090146
:1018900012099942FBD9430801E0490052089942D4
:1018A000FBD900E04908401A07D35241FAD3014658
:1018B0001046704749084018F7D29218FAD34018DA
:1018C000014610467047CB0F00D04942021000D5A8
:1018D0004042534008B5FFF7D4FF0CBC521000D370
:1018E0004042002A00D549421847F446002000F043
:1018F0002EF86047F0B517001F4323D00126440897
:10190000CF073C434D08A71A2F469F4103D3921897
:101910005B410136F7E70024002505E05208DF07A8
:101920003A435B0824196D41871A0F469F4102D341
:10193000801A99410134013EF0D102460B462046FF
:101940002946F0BD0020002100F001F8F0BD7047ED
:1019500010B580249E23C10D0202240622435B1A87
:1019600002D4DA40101C06E0FE2902D90020A2426F
:1019700001D1090A481E10BD00282BD0030C01D14B
:10198000000402E080231B05C918030E01D10002E8
:1019900002E08023DB04C918030F01D1000102E03B
:1019A00080239B04C918830F01D1800002E08023AB
:1019B0005B04C918002801DB400002E080231B04FF
:1019C000C918803003125918000601D10123994328
:1019D000081C00E000207047802108B5C905FFF70A
:1019E000CBFF08BD8446830708D18B0706D1131FA0
:1019F00004D304C904C0043BFBD21A1D524205D0D3
:101A0000891A801A8B5C83540132FBD1604670477F
:101A10008446043A09D3830707D109060B0A194300
:101A20000B0C1943043A02C0FCD2043203D00170FB
:101A30000130013AFBD1604670478C46714601394E
:101A4000095C49008E446146704738433137313173
:101A50002D3838636430303030000000001BB70090
:101A60000000000000000000C027090090051000E1
:101A7000C05C1500F0B31A00200B2000009F24006A
:101A8000E0322900C0C62D0050973100E0673500D4
:101A90007038390000093D004016400080234300A3
:101AA000C03046000C000C00C00000000300010024
:101AB0000C000600C0000000030002000C0004003F
:101AC000C0000000030003000C000300C000000081
:101AD000030004000C000200C00000000300060028
:101AE0000C000100C000000003000C0018001800EA
:101AF000C00001000200010018000C00C00001003D
:101B00000200020018000800C000010002000300EB
:101B100018000600C00001000200040018000400C4
:101B2000C00001000200060018000300C000010010
:101B30000200080018000200C000010002000C00B2
:101B400018000100C000010002001800240012006B
:101B5000200102000200020024000C00200102000B
:101B6000020003002400090020010200020004001A
:101B700024000600200102000200060024000400E8
:101B800020010200020009002400030020010200DD
:101B900002000C00240002002001020002001200DA
:101BA000240001002001020002002400300018007F
:101BB000C00003000100020030001000C00003005C
:101BC0000100030030000C00C0000300010004000D
:101BD00030000800C00003000100060030000600CD
:101BE000C00003000100080030000400C000030032
:101BF00001000C0030000300C000030001001000D1
:101C000030000200C0000300010018003000010095
:101C1000C0000300010030003C001E00F000040082
:101C2000010002003C001400F00004000100030069
:101C30003C000F00F0000400010004003C000C0018
:101C4000F0000400010005003C000A00F000040060
:101C5000010006003C000600F000040001000A003C
:101C60003C000500F000040001000C003C000400F2
:101C7000F000040001000F003C000300F00004002D
:101C8000010014003C000200F000040001001E00EE
:101C90003C000100F000040001003C004800180076
:101CA000200105000100030048001200200105008A
:101CB0000100040048000C0020010500010006009E
:101CC0004800090020010500010008004800080044
:101CD0002001050001000900480006002001050060
:101CE00001000C0048000400200105000100120062
:101CF0004800030020010500010018004800020010
:101D00002001050001002400480001002001050019
:101D10000100480054001C00A80006000000030059
:101D200054001500A80006000000040054000E0036
:101D3000A80006000000060054000C00A8000600E1
:101D40000000070054000700A800060000000C0077
:101D500054000600A800060000000E005400040015
:101D6000A80006000000150054000300A8000600AB
:101D700000001C0054000200A800060000002A0019
:101D800054000100A8000600000054006000180084
:101D9000C00007000000040060001000C000070041
:101DA0000000060060000C00C000070000000800F2
:101DB00060000800C000070000000C006000060082
:101DC000C00007000000100060000400C000070011
:101DD0000000180060000300C000070000002000A1
:101DE00060000200C0000700000030006000010039
:081DF000C000070000006000C4
:0400000300000103F5
:00000001FF
